:020000040000FA
:0400000003303A2867
:08000800A000030EA100831209
:1000100005191028831601178312B23081002B288E
:1000200083160113831203140B190310A80DA90DD5
:10003000AA0DAB0DAC0DAC16FF302C02031D2B2806
:10004000FA302B02031D2B2831152A08AF0029088E
:10005000AE002808AD008B100B11210E8300A00EFE
:04006000200E090065
:0C007400203084008001840A6030040207
:10008000031C3C281230B00098218316FF239000F7
:10009000831283160C308505870183128501870141
:1000A000073099000030831691009F008312C830FA
:1000B00083168100831231309000003083168C004B
:1000C000831210308B00831600309B001C141A081A
:1000D0008312BC00851DD321831610309B001C1495
:1000E0001A088312BD00CB2181018E018F010B11F3
:1000F0008B100B108C018B178B2031198E20B30BBA
:100100008928031085190314B90DF0303902031939
:100110001321F8217C2864003210080031110130CD
:10012000B7008B132030370783169B001C141A0866
:100130008312A4001030370783169B001C141A0882
:100140008312A300A6000230A606003037078316EC
:100150009B001C141A088312A200A7000130A706F6
:100160008B17321CB92822090339A200A309A4095C
:10017000A50924082F02031D0D2923082E02031DA3
:100180000D2922082D02031D0D2901303702031D00
:10019000CE283D18CE283D143E149F210230370250
:1001A000031DD728BD18D728BD143E14A321033042
:1001B0003702031DE0283D19E0283D153E14A72114
:1001C00004303702031DE928BD19E928BD153E1486
:1001D000AB2105303702031DF2283D1AF2283D16E7
:1001E0003E14AF2106303702031DFB28BD1AFB2841
:1001F000BD163E14B02107303702031D04293D1BF4
:1002000004293D173E14B12108303702031D0D2982
:10021000BD1B0D29BD173E14B221B70A05303702A8
:100220000318080091280130B600B300B400B500EF
:10023000B70085018701B1138B20B30B4B29031045
:1002400085190314B90DF030390203197229B40B62
:100250004B29013037020319B32102303702031949
:10026000B721033037020319BB21043037020319C9
:10027000C321053037020319C7210630370203199D
:10028000C821073037020319C92108303702031982
:10029000CA219630B400311D1C293111321C552958
:1002A0002D090339AD00AE09AF092F1C1C298E01A1
:1002B0008F010C1C1C290C102E1E1C298B132030A6
:1002C0003707BB002F08BA00852110303707BB0065
:1002D0002E08BA00852100303707BB002D08BA0070
:1002E00085218B1785018701B70AB60105303702D2
:1002F000031C1C29CB2108003E1C08003E101030B6
:10030000BB003D08BA00852108008B133A0883160C
:100310001C159A003B089B0055309D00AA309D009B
:100320009C1464009C1891291C1183128B170800DF
:10033000FF30D000D415D515D615D71508000330D9
:10034000D204BD1008000330D2043D1008000C3068
:10035000D204BD1108000C30D2043D110800080081
:100360000800080008000508023A85000800050892
:10037000013A850008000C308316850083120508B9
:10038000203A850008000508103A8500080008009A
:100390000800080008003D08D200031D08000530D1
:1003A000BD00D2000800B601B301B4013C1CDB293A
:1003B000BC01BC14DD29BC013C143C08B60064003F
:1003C000E129E229E329E429E529B41B8514B41FB6
:1003D0008510B30BDF29B40BDF290310B60CB60868
:1003E000031DDF290030BB003C08BA00852108004E
:1003F0008F08031908008F01D00F992AD00A023004
:100400005205031D122A541D082AD4015416202A0D
:10041000D41D0D2AD4015416202A541E202AD4019A
:10042000D414202AD41C172AD4015415202A541D70
:100430001C2AD401D415202A541E202AD401541574
:1004400001305205031D332A551D292AD5015516A1
:10045000412AD51D2E2AD5015516412A551E412A5D
:10046000D501D514412AD51C382AD5015515412A64
:10047000551D3D2AD501D515412A551E412AD501C4
:1004800055150830BC180A305205031D562A561D52
:100490004C2AD6015616642AD61D512AD601561664
:1004A000642A561E642AD601D614642AD61C5B2AF6
:1004B000D6015615642A561D602AD601D615642A1F
:1004C000561E642AD60156150430BC180630520553
:1004D000031D792A571D6F2AD7015716872AD71D62
:1004E000742AD7015716872A571E872AD701D7148F
:1004F000872AD71C7E2AD7015715872A571D832A9A
:10050000D701D715872A571E872AD7015715BC1C34
:10051000922AD21C922AD51C922A3C30831685003E
:100520008312962A0C308316850083127C213D08A5
:10053000D2005008D1000C305405031D85100C303A
:100540005505031D05100C305605031D85120C3092
:100550005705031D051251080E020318C32A123055
:100560005405031D851412305505031D0514123062
:100570005605031D851612305705031D0516FF305D
:100580005002031908008F08031D08008B20510832
:100590000E02031CC32A18305405031D85100630B3
:1005A0005405031D851418305505031D051006302C
:1005B0005505031D051418305605031D8512063018
:1005C0005605031D851618305705031D0512063004
:0805D0005705031D0516080084
:084000000200030003000800A8
:02400E00CC01E3
:10420000010078007A007C007E007B0079007F004E
:104210007D007A0078007E007C00FF00FF00FF0038
:104220000000F200F600FA00FE00F200F600FA00CC
:10423000FE00F200F600FA00FE00FF00FF00FF00A3
:10424000010005000500050005000900090009003E
:1042500009000D000D000D000D00FF00FF00FF0024
:10426000FF00FF00FF00FF00FF00FF00FF00FF0056
:10427000FF00FF00FF00FF00FF00FF00FF00FF0046
:10428000FF00FF00FF00FF00FF00FF00FF00FF0036
:10429000FF00FF00FF00FF00FF00FF00FF00FF0026
:1042A000FF00FF00FF00FF00FF00FF00FF00FF0016
:1042B000FF00FF00FF00FF00FF00FF00FF00FF0006
:1042C000FF00FF00FF00FF00FF00FF00FF00FF00F6
:1042D000FF00FF00FF00FF00FF00FF00FF00FF00E6
:1042E000FF00FF00FF00FF00FF00FF00FF00FF00D6
:1042F000FF00FF00FF00FF00FF00FF00FF00DD00E8
:00000001FF
